ARM Linker, RVCT3.1 [Build 903] for uVision [Professional]

================================================================================

Section Cross References

    __main.o(!!!main) refers to kernel.o(.text) for __rt_entry
    kernel.o(.text) refers to stkheap1.o(.text) for __rt_stackheap_init
    kernel.o(.text) refers to boardinit2.o(.text) for _platform_post_stackheap_init
    kernel.o(.text) refers to lib_init.o(.text) for __rt_lib_init
    kernel.o(.text) refers to boardinit3.o(.text) for _platform_post_lib_init
    kernel.o(.text) refers to exit.o(.text) for exit
    kernel.o(.text) refers to c_call.o(.text) for main
    kernel.o(.text) refers to sys_exit.o(.text) for _sys_exit
    kernel.o(.ARM.exidx) refers to kernel.o(.text) for __rt_entry
    sys_exit.o(.text) refers to use_no_semi.o(.text) for __I_use_semihosting
    exit.o(.text) refers to kernel.o(.text) for __rt_exit
    stkheap1.o(.text) refers to sys_stackheap_outer.o(.text) for __user_setup_stackheap
    stkheap1.o(.text) refers to rt_stackheap_storage_intlibspace.o(.text) for __rt_stackheap_storage
    stkheap2.o(.text) refers to sys_stackheap_outer.o(.text) for __user_setup_stackheap
    stkheap2.o(.text) refers to rt_stackheap_storage_intlibspace.o(.text) for __rt_stackheap_storage
    lib_init.o(.emb_text) refers to no_argv.o(.text) for __ARM_get_argv
    lib_init.o(.text) refers to fpinit.o(x$fpl$fpinit) for _fp_init
    lib_init.o(.text) refers to lib_init.o(.emb_text) for __ARM_argv_veneer
    lib_init.o(.text) refers to rt_locale_intlibspace.o(.text) for __rt_locale
    sys_stackheap_outer.o(.text) refers to libspace.o(.text) for __user_perproc_libspace
    sys_stackheap_outer.o(.text) refers to sys_stackheap.o(.text) for __user_initial_stackheap
    rt_stackheap_storage.o(.text) refers to rt_stackheap_storage.o(.bss) for __rt_stackheap_storage_data
    rt_stackheap_storage_intlibspace.o(.text) refers (Weak) to libspace.o(.bss) for __libspace_start
    rt_stackheap_storage_onelibspace.o(.text) refers (Weak) to libspace.o(.text) for __user_libspace
    rt_stackheap_storage_twolibspace.o(.text) refers (Weak) to libspace.o(.text) for __user_perproc_libspace
    rt_locale.o(.text) refers to rt_locale.o(.bss) for __rt_locale_data
    rt_locale_intlibspace.o(.text) refers (Weak) to libspace.o(.bss) for __libspace_start
    rt_locale_onelibspace.o(.text) refers (Weak) to libspace.o(.text) for __user_libspace
    rt_locale_twolibspace.o(.text) refers (Weak) to libspace.o(.text) for __user_perproc_libspace
    _get_argv.o(.text) refers to heapext.o(.text) for __heap_extend
    _get_argv.o(.text) refers to defsig_rtmem_outer.o(.text) for __rt_SIGRTMEM
    _get_argv.o(.text) refers to sys_command.o(.text) for _sys_command_string
    _get_argv.o(.text) refers (Special) to hrguard.o(.text) for __heap_region_guard
    fpinit.o(x$fpl$fpinit) refers to rt_fp_status_addr_intlibspace.o(.text) for __rt_fp_status_addr
    sys_command.o(.text) refers (Special) to use_no_semi.o(.text) for __I_use_semihosting
    sys_stackheap.o(.text) refers to use_no_semi.o(.text) for __I_use_semihosting
    libspace.o(.text) refers to libspace.o(.bss) for __libspace_start
    rt_fp_status_addr.o(.text) refers to rt_fp_status_addr.o(.bss) for __rt_fp_status_addr_data
    rt_fp_status_addr_intlibspace.o(.text) refers (Weak) to libspace.o(.bss) for __libspace_start
    rt_fp_status_addr_onelibspace.o(.text) refers (Weak) to libspace.o(.text) for __user_libspace
    rt_fp_status_addr_twolibspace.o(.text) refers (Weak) to libspace.o(.text) for __user_perthread_libspace
    defsig_rtmem_outer.o(.text) refers to defsig_rtmem_inner.o(.text) for __rt_SIGRTMEM_inner
    defsig_rtmem_outer.o(.text) refers to defsig_exit.o(.text) for __sig_exit
    defsig_rtmem_formal.o(.text) refers to rt_raise.o(.text) for __rt_raise
    defsig_rtmem_formal.o(.text) refers (Special) to defsig_rtmem_inner.o(.text) for __rt_SIGRTMEM_inner
    heapext.o(.text) refers to stkheap1.o(.text) for __rt_heap_extend
    rt_raise.o(.text) refers to __raise.o(.text) for __raise
    rt_raise.o(.text) refers to sys_exit.o(.text) for _sys_exit
    defsig_exit.o(.text) refers to sys_exit.o(.text) for _sys_exit
    defsig_rtmem_inner.o(.text) refers to defsig_general.o(.text) for __default_signal_display
    __raise.o(.text) refers to defsig.o(CL$$defsig) for __default_signal_handler
    defsig_general.o(.text) refers to sys_wrch.o(.text) for _ttywrch
    sys_wrch.o(.text) refers (Special) to use_no_semi.o(.text) for __I_use_semihosting
    defsig.o(CL$$defsig) refers (Weak) to defsig_rtmem_inner.o(.text) for __rt_SIGRTMEM_inner


================================================================================

Image Symbol Table

    Local Symbols

    Symbol Name                              Value     Ov Type        Size  Object(Section)

    ../../angel/boardlib.s                   0x00000000   Number         0  cpuinit.o ABSOLUTE
    ../../angel/boardlib.s                   0x00000000   Number         0  boardinit1.o ABSOLUTE
    ../../angel/boardlib.s                   0x00000000   Number         0  boardinit2.o ABSOLUTE
    ../../angel/boardlib.s                   0x00000000   Number         0  boardshut.o ABSOLUTE
    ../../angel/boardlib.s                   0x00000000   Number         0  boardinit3.o ABSOLUTE
    ../../angel/handlers.s                   0x00000000   Number         0  __scatter_zi.o ABSOLUTE
    ../../angel/kernel.s                     0x00000000   Number         0  kernel.o ABSOLUTE
    ../../angel/rt.s                         0x00000000   Number         0  rt_locale.o ABSOLUTE
    ../../angel/rt.s                         0x00000000   Number         0  rt_fp_status_addr_twolibspace.o ABSOLUTE
    ../../angel/rt.s                         0x00000000   Number         0  rt_locale_intlibspace.o ABSOLUTE
    ../../angel/rt.s                         0x00000000   Number         0  rt_fp_status_addr_onelibspace.o ABSOLUTE
    ../../angel/rt.s                         0x00000000   Number         0  rt_fp_status_addr_intlibspace.o ABSOLUTE
    ../../angel/rt.s                         0x00000000   Number         0  rt_raise.o ABSOLUTE
    ../../angel/rt.s                         0x00000000   Number         0  rt_fp_status_addr.o ABSOLUTE
    ../../angel/rt.s                         0x00000000   Number         0  rt_locale_twolibspace.o ABSOLUTE
    ../../angel/rt.s                         0x00000000   Number         0  rt_stackheap_storage.o ABSOLUTE
    ../../angel/rt.s                         0x00000000   Number         0  rt_stackheap_storage_intlibspace.o ABSOLUTE
    ../../angel/rt.s                         0x00000000   Number         0  rt_locale_onelibspace.o ABSOLUTE
    ../../angel/rt.s                         0x00000000   Number         0  rt_stackheap_storage_onelibspace.o ABSOLUTE
    ../../angel/rt.s                         0x00000000   Number         0  rt_stackheap_storage_twolibspace.o ABSOLUTE
    ../../angel/scatter.s                    0x00000000   Number         0  __scatter.o ABSOLUTE
    ../../angel/startup.s                    0x00000000   Number         0  __main.o ABSOLUTE
    ../../angel/sys.s                        0x00000000   Number         0  sys_exit.o ABSOLUTE
    ../../angel/sys.s                        0x00000000   Number         0  libspace.o ABSOLUTE
    ../../angel/sys.s                        0x00000000   Number         0  sys_stackheap.o ABSOLUTE
    ../../angel/sys.s                        0x00000000   Number         0  use_no_semi.o ABSOLUTE
    ../../angel/sys.s                        0x00000000   Number         0  sys_stackheap_outer.o ABSOLUTE
    ../../angel/sysapp.c                     0x00000000   Number         0  sys_command.o ABSOLUTE
    ../../angel/sysapp.c                     0x00000000   Number         0  sys_wrch.o ABSOLUTE
    ../../armsys.c                           0x00000000   Number         0  lib_init.o ABSOLUTE
    ../../armsys.c                           0x00000000   Number         0  lib_init.o ABSOLUTE
    ../../armsys.c                           0x00000000   Number         0  _get_argv.o ABSOLUTE
    ../../armsys.c                           0x00000000   Number         0  no_argv.o ABSOLUTE
    ../../fpinit.s                           0x00000000   Number         0  fpinit.o ABSOLUTE
    ../../heapalloc.c                        0x00000000   Number         0  hrguard.o ABSOLUTE
    ../../signal.c                           0x00000000   Number         0  defsig_rtmem_inner.o ABSOLUTE
    ../../signal.c                           0x00000000   Number         0  defsig_rtmem_formal.o ABSOLUTE
    ../../signal.c                           0x00000000   Number         0  defsig_exit.o ABSOLUTE
    ../../signal.c                           0x00000000   Number         0  defsig_rtmem_outer.o ABSOLUTE
    ../../signal.c                           0x00000000   Number         0  defsig_general.o ABSOLUTE
    ../../signal.c                           0x00000000   Number         0  __raise.o ABSOLUTE
    ../../signal.s                           0x00000000   Number         0  defsig.o ABSOLUTE
    ../../stdlib.c                           0x00000000   Number         0  exit.o ABSOLUTE
    ../../stkheap.s                          0x00000000   Number         0  heapext.o ABSOLUTE
    ../../stkheap1.s                         0x00000000   Number         0  stkheap1.o ABSOLUTE
    ../../stkheap2.s                         0x00000000   Number         0  stkheap2.o ABSOLUTE
    C_CALL.C                                 0x00000000   Number         0  c_call.o ABSOLUTE
    dc.s                                     0x00000000   Number         0  dc.o ABSOLUTE
    !!!main                                  0x30000000   Section        8  __main.o(!!!main)
    !!!scatter                               0x30000008   Section       60  __scatter.o(!!!scatter)
    !!handler_zi                             0x30000044   Section       44  __scatter_zi.o(!!handler_zi)
    .emb_text                                0x30000070   Section       16  lib_init.o(.emb_text)
    .text                                    0x30000080   Section       72  c_call.o(.text)
    .text                                    0x300000c8   Section      104  kernel.o(.text)
    .text                                    0x30000130   Section       24  sys_exit.o(.text)
    .text                                    0x30000148   Section       12  exit.o(.text)
    .text                                    0x30000154   Section      152  stkheap1.o(.text)
    .text                                    0x300001ec   Section      194  lib_init.o(.text)
    .text                                    0x300002b0   Section       12  boardinit2.o(.text)
    .text                                    0x300002bc   Section       16  boardinit3.o(.text)
    .text                                    0x300002cc   Section        4  use_no_semi.o(.text)
    .text                                    0x300002d0   Section       96  sys_stackheap_outer.o(.text)
    .text                                    0x30000330   Section       16  rt_stackheap_storage_intlibspace.o(.text)
    .text                                    0x30000340   Section       16  rt_locale_intlibspace.o(.text)
    .text                                    0x30000350   Section        2  no_argv.o(.text)
    .text                                    0x30000354   Section       80  sys_stackheap.o(.text)
    .text                                    0x300003a4   Section       12  libspace.o(.text)
    .text                                    0x300003b0   Section       16  rt_fp_status_addr_intlibspace.o(.text)
    x$fpl$fpinit                             0x300003c0   Section       24  fpinit.o(x$fpl$fpinit)
    .bss                                     0x300003e8   Section       96  libspace.o(.bss)

    Global Symbols

    Symbol Name                              Value     Ov Type        Size  Object(Section)

    BuildAttributes$$THM_ISAv2$ARM_ISAv5$M$E$P$S$PE$A:L22$X:L11$S22$IEEE1$IW$USESV6$~STKCKD$USESV7$~SHL$OSPACE$EBA8$STANDARDLIB$REQ8$PRES8$EABIv2 0x00000000   Number         0  anon$$obj.o ABSOLUTE
    __ARM_use_no_argv                        0x00000000   Number         0  c_call.o ABSOLUTE
    __ARM_exceptions_init                     - Undefined Weak Reference
    __Heap_DescSize                           - Undefined Weak Reference
    __alloca_initialize                       - Undefined Weak Reference
    __cpp_initialize__aeabi_                  - Undefined Weak Reference
    __cxa_finalize                            - Undefined Weak Reference
    __rt_SIGABRT_inner                        - Undefined Weak Reference
    __rt_SIGCPPL_inner                        - Undefined Weak Reference
    __rt_SIGFPE_inner                         - Undefined Weak Reference
    __rt_SIGILL_inner                         - Undefined Weak Reference
    __rt_SIGINT_inner                         - Undefined Weak Reference
    __rt_SIGPVFN_inner                        - Undefined Weak Reference
    __rt_SIGRTRED_inner                       - Undefined Weak Reference
    __rt_SIGSEGV_inner                        - Undefined Weak Reference
    __rt_SIGSTAK_inner                        - Undefined Weak Reference
    __rt_SIGTERM_inner                        - Undefined Weak Reference
    __rt_SIGUSR1_inner                        - Undefined Weak Reference
    __rt_SIGUSR2_inner                        - Undefined Weak Reference
    __rt_sigother_inner                       - Undefined Weak Reference
    __sigvec_lookup                           - Undefined Weak Reference
    __user_heap_extend                        - Undefined Weak Reference
    _atexit_init                              - Undefined Weak Reference
    _call_atexit_fns                          - Undefined Weak Reference
    _clock_init                               - Undefined Weak Reference
    _fp_trap_init                             - Undefined Weak Reference
    _get_lc_collate                           - Undefined Weak Reference
    _get_lc_ctype                             - Undefined Weak Reference
    _get_lc_monetary                          - Undefined Weak Reference
    _get_lc_numeric                           - Undefined Weak Reference
    _get_lc_time                              - Undefined Weak Reference
    _getenv_init                              - Undefined Weak Reference
    _handle_redirection                       - Undefined Weak Reference
    _init_alloc                               - Undefined Weak Reference
    _init_user_alloc                          - Undefined Weak Reference
    _initio                                   - Undefined Weak Reference
    _rand_init                                - Undefined Weak Reference
    _signal_init                              - Undefined Weak Reference
    _terminate_user_alloc                     - Undefined Weak Reference
    _terminateio                              - Undefined Weak Reference
    __main                                   0x30000000   ARM Code       8  __main.o(!!!main)
    __scatterload                            0x30000008   ARM Code       0  __scatter.o(!!!scatter)
    __scatterload_rt2                        0x30000008   ARM Code      52  __scatter.o(!!!scatter)
    __scatterload_null                       0x3000001c   ARM Code       0  __scatter.o(!!!scatter)
    __scatterload_zeroinit                   0x30000044   ARM Code      44  __scatter_zi.o(!!handler_zi)
    __ARM_argv_veneer                        0x30000070   ARM Code      16  lib_init.o(.emb_text)
    delay                                    0x30000080   ARM Code      48  c_call.o(.text)
    main                                     0x300000b0   ARM Code      24  c_call.o(.text)
    __rt_entry                               0x300000c8   ARM Code      76  kernel.o(.text)
    __rt_exit                                0x30000114   ARM Code      20  kernel.o(.text)
    __rt_abort                               0x30000128   ARM Code       8  kernel.o(.text)
    _sys_exit                                0x30000130   ARM Code      20  sys_exit.o(.text)
    exit                                     0x30000149   Thumb Code    12  exit.o(.text)
    __rt_stackheap_init                      0x30000154   ARM Code      40  stkheap1.o(.text)
    __rt_heap_extend                         0x3000017c   ARM Code     112  stkheap1.o(.text)
    __rt_lib_init                            0x300001ed   Thumb Code   176  lib_init.o(.text)
    __rt_lib_shutdown                        0x3000029d   Thumb Code    18  lib_init.o(.text)
    _platform_post_stackheap_init            0x300002b0   ARM Code      12  boardinit2.o(.text)
    _platform_post_lib_init                  0x300002bc   ARM Code      16  boardinit3.o(.text)
    __I_use_semihosting                      0x300002cc   ARM Code       0  use_no_semi.o(.text)
    __use_no_semihosting_swi                 0x300002cc   ARM Code       4  use_no_semi.o(.text)
    __user_setup_stackheap                   0x300002d0   ARM Code      96  sys_stackheap_outer.o(.text)
    __rt_stackheap_storage                   0x30000330   ARM Code      12  rt_stackheap_storage_intlibspace.o(.text)
    __rt_locale                              0x30000340   ARM Code      12  rt_locale_intlibspace.o(.text)
    __ARM_get_argv                           0x30000351   Thumb Code     2  no_argv.o(.text)
    __user_initial_stackheap                 0x30000354   ARM Code      80  sys_stackheap.o(.text)
    _RW_Limit                                0x300003a0   Data           0  sys_stackheap.o(.text)
    __user_libspace                          0x300003a4   ARM Code       8  libspace.o(.text)
    __user_perproc_libspace                  0x300003a4   ARM Code       0  libspace.o(.text)
    __user_perthread_libspace                0x300003a4   ARM Code       0  libspace.o(.text)
    __rt_fp_status_addr                      0x300003b0   ARM Code      12  rt_fp_status_addr_intlibspace.o(.text)
    _fp_init                                 0x300003c0   ARM Code      24  fpinit.o(x$fpl$fpinit)
    __fplib_config_pureend_doubles           0x300003d0   ARM Code       0  fpinit.o(x$fpl$fpinit)
    Region$$Table$$Base                      0x300003d8   Number         0  anon$$obj.o(Region$$Table)
    Region$$Table$$Limit                     0x300003e8   Number         0  anon$$obj.o(Region$$Table)
    __libspace_start                         0x300003e8   Data          96  libspace.o(.bss)
    Image$$ZI$$Limit                         0x30000448   Number         0  anon$$obj.o(linker$$defined$$symbols)
    __temporary_stack_top_libspace           0x30000448   Number         0  libspace.o(.bss)


================================================================================

Memory Map of the image

  Image Entry point : 0x30000000

  Load Region LR_1 (Base: 0x30000000, Size: 0x000003e8, Max: 0xffffffff, ABSOLUTE)

    Execution Region ER_RO (Base: 0x30000000, Size: 0x000003e8, Max: 0xffffffff, ABSOLUTE)

    Base Addr    Size         Type   Attr      Idx    E Section Name        Object

    0x30000000   0x00000008   Code   RO           18  * !!!main             __main.o(c_5.l)
    0x30000008   0x0000003c   Code   RO          113    !!!scatter          __scatter.o(c_5.l)
    0x30000044   0x0000002c   Code   RO          115    !!handler_zi        __scatter_zi.o(c_5.l)
    0x30000070   0x00000010   Code   RO           31    .emb_text           lib_init.o(c_5.l)
    0x30000080   0x00000048   Code   RO            1    .text               c_call.o
    0x300000c8   0x00000068   Code   RO           20    .text               kernel.o(c_5.l)
    0x30000130   0x00000018   Code   RO           23    .text               sys_exit.o(c_5.l)
    0x30000148   0x0000000c   Code   RO           25    .text               exit.o(c_5.l)
    0x30000154   0x00000098   Code   RO           27    .text               stkheap1.o(c_5.l)
    0x300001ec   0x000000c2   Code   RO           32    .text               lib_init.o(c_5.l)
    0x300002ae   0x00000002   PAD
    0x300002b0   0x0000000c   Code   RO           37    .text               boardinit2.o(c_5.l)
    0x300002bc   0x00000010   Code   RO           39    .text               boardinit3.o(c_5.l)
    0x300002cc   0x00000004   Code   RO           43    .text               use_no_semi.o(c_5.l)
    0x300002d0   0x00000060   Code   RO           45    .text               sys_stackheap_outer.o(c_5.l)
    0x30000330   0x00000010   Code   RO           50    .text               rt_stackheap_storage_intlibspace.o(c_5.l)
    0x30000340   0x00000010   Code   RO           59    .text               rt_locale_intlibspace.o(c_5.l)
    0x30000350   0x00000002   Code   RO           69    .text               no_argv.o(c_5.l)
    0x30000352   0x00000002   PAD
    0x30000354   0x00000050   Code   RO           75    .text               sys_stackheap.o(c_5.l)
    0x300003a4   0x0000000c   Code   RO           77    .text               libspace.o(c_5.l)
    0x300003b0   0x00000010   Code   RO           83    .text               rt_fp_status_addr_intlibspace.o(c_5.l)
    0x300003c0   0x00000018   Code   RO           71    x$fpl$fpinit        fpinit.o(fz_5s.l)
    0x300003d8   0x00000010   Data   RO          111    Region$$Table       anon$$obj.o


    Execution Region ER_RW (Base: 0x300003e8, Size: 0x00000000, Max: 0xffffffff, ABSOLUTE)

    **** No section assigned to this execution region ****


    Execution Region ER_ZI (Base: 0x300003e8, Size: 0x00000060, Max: 0xffffffff, ABSOLUTE)

    Base Addr    Size         Type   Attr      Idx    E Section Name        Object

    0x300003e8   0x00000060   Zero   RW           78    .bss                libspace.o(c_5.l)


================================================================================

Image component sizes


      Code (inc. data)   RO Data    RW Data    ZI Data      Debug   Object Name

        72          0          0          0          0       2889   c_call.o

    ------------------------------------------------------------------------
        72          0         16          0          0       2892   Object Totals
         0          0         16          0          0          0   (incl. Generated)
         0          0          0          0          0          3   (incl. Padding)

    ------------------------------------------------------------------------

      Code (inc. data)   RO Data    RW Data    ZI Data      Debug   Library Member Name

         8          0          0          0          0          0   __main.o
        60          8          0          0          0          0   __scatter.o
        44          0          0          0          0          0   __scatter_zi.o
        12          0          0          0          0          0   boardinit2.o
        16          0          0          0          0          0   boardinit3.o
        12          0          0          0          0          0   exit.o
        24          0          0          0          0          0   fpinit.o
       104          4          0          0          0          0   kernel.o
       210          4          0          0          0          0   lib_init.o
        12          4          0          0         96          0   libspace.o
         2          0          0          0          0          0   no_argv.o
        16          4          0          0          0          0   rt_fp_status_addr_intlibspace.o
        16          4          0          0          0          0   rt_locale_intlibspace.o
        16          4          0          0          0          0   rt_stackheap_storage_intlibspace.o
       152          0          0          0          0          0   stkheap1.o
        24          8          0          0          0          0   sys_exit.o
        80          8          0          0          0          0   sys_stackheap.o
        96          0          0          0          0          0   sys_stackheap_outer.o
         4          0          0          0          0          0   use_no_semi.o

    ------------------------------------------------------------------------
       912         48          0          0         96          0   Library Totals
         4          0          0          0          0          0   (incl. Padding)

    ------------------------------------------------------------------------

      Code (inc. data)   RO Data    RW Data    ZI Data      Debug   Library Name

       884         48          0          0         96          0   c_5.l
        24          0          0          0          0          0   fz_5s.l

    ------------------------------------------------------------------------
       912         48          0          0         96          0   Library Totals

    ------------------------------------------------------------------------

================================================================================


      Code (inc. data)   RO Data    RW Data    ZI Data      Debug   

       984         48         16          0         96       2892   Grand Totals
       984         48         16          0         96       2892   ELF Image Totals
       984         48         16          0          0          0   ROM Totals

================================================================================

    Total RO  Size (Code + RO Data)                 1000 (   0.98kB)
    Total RW  Size (RW Data + ZI Data)                96 (   0.09kB)
    Total ROM Size (Code + RO Data + RW Data)       1000 (   0.98kB)

================================================================================

